:100000008316043085000030860083127D2800307E
:1000100091000030920008309300003094000030CE
:1000200095003E28003091001C309200143093005F
:100030001C309400003095003E283E309100223064
:10004000920022309300223094003E3095003E28EA
:100050004130910041309200413093004130940092
:10006000413095003E280030910000309200003071
:10007000930000309400003095003E288514000065
:10008000851011088600512012088600512013089F
:100090008600512014088600512015088600512042
:1000A0000800051955281E1256281E169B0B5628A7
:1000B00000308600051400000510051D08001E1AFA
:1000C00008009E12080050308C0007208C0B652819
:1000D00010308C0012208C0B6A2810308C001D20F0
:1000E0008C0B6F2810308C0028208C0B7428083063
:1000F0008C0033208C0B792808009E121E12051DDF
:1001000084289E1663207F289E1E7F2863207F28D8
:00000001FF
